:0200000480007A
:100000006F008004732F2034930F80006308FF0378
:10001000930F90006304FF03930FB0006300FF038E
:10002000130F000063040F0067000F00732F2034CC
:1000300063540F006F00400093E19153171F0000BD
:1000400023223FFC6FF09FFF93000000130100008C
:10005000930100001302000093020000130300004C
:100060009303000013040000930400001305000034
:10007000930500001306000093060000130700001C
:100080009307000013080000930800001309000004
:1000900093090000130A0000930A0000130B0000EC
:1000A000930B0000130C0000930C0000130D0000D4
:1000B000930D0000130E0000930E0000130F0000BC
:1000C000930F0000732540F16310050097020000B4
:1000D000938202017390523073500018970200000F
:1000E00093824202739052309B021000939252030B
:1000F0009382F2FF7390023B9302F0017390023AF5
:100100007350403097020000938242017390523046
:10011000735020307350303093010000970200007C
:10012000938282EE73905230130510001315F5017F
:10013000635C05000F00F00F930110009308D005D9
:10014000130500007300000093020000638A0200A0
:1001500073905210B7B200009B82921073902230BD
:100160007350003097020000938242017390123462
:10017000732540F17300203093000000130100004C
:100180003B87200293030000930120006312773C19
:1001900093001000130110003B872002930310000E
:1001A000930130006316773A93003000130170001A
:1001B0003B8720029303500193014000631A773874
:1001C000930000003781FFFF3B872002930300006C
:1001D00093015000631E7736B700008013010000C2
:1001E0003B8720029303000093016000631277367F
:1001F000B70000803781FFFF3B8720029303000098
:1002000093017000631677349300D0001301B0009F
:10021000BB8020029303F00893018000639A703240
:100220009300E0001301B0003B8120029303A0097A
:1002300093019000631E71309300D000BB801002C8
:100240009303900A9301A00063947030130200009E
:100250009300D0001301B0003B8720021303070076
:100260001302120093022000E31452FE9303F008DD
:100270009301B000631E732C130200009300E00092
:100280001301B0003B872002130000001303070096
:100290001302120093022000E31252FE9303A009FE
:1002A0009301C0006316732A130200009300F0004C
:1002B0001301B0003B872002130000001300000070
:1002C000130307001302120093022000E31052FEF2
:1002D0009303500A9301D000631C7326130200009D
:1002E0009300D0001301B0003B87200213021200DC
:1002F00093022000E31652FE9303F0089301E000FE
:1003000063187724130200009300E0001301B0008B
:10031000130000003B87200213021200930220000A
:10032000E31452FE9303A0099301F00063127722B5
:10033000130200009300F0001301B000130000004E
:10034000130000003B8720021302120093022000DA
:10035000E31252FE9303500A93010001631A771EC1
:10036000130200009300D000130000001301B0003E
:100370003B8720021302120093022000E31452FE76
:100380009303F008930110016314771C130200001B
:100390009300E000130000001301B0001300000000
:1003A0003B8720021302120093022000E31252FE48
:1003B0009303A00993012001631C77181302000026
:1003C0009300F00013000000130000001301B000C0
:1003D0003B8720021302120093022000E31252FE18
:1003E0009303500A9301300163147716130200003F
:1003F0001301B0009300D0003B87200213021200CB
:1004000093022000E31652FE9303F008930140018B
:1004100063107714130200001301B0009300E00092
:10042000130000003B8720021302120093022000F9
:10043000E31452FE9303A00993015001631A77104D
:10044000130200001301B0009300F000130000003D
:10045000130000003B8720021302120093022000C9
:10046000E31252FE9303500A930160016312770E68
:10047000130200001301B000130000009300D0002D
:100480003B8720021302120093022000E31452FE65
:100490009303F00893017001631C770A13020000B4
:1004A0001301B000130000009300E00013000000EF
:1004B0003B8720021302120093022000E31252FE37
:1004C0009303A009930180016314770813020000CD
:1004D0001301B00013000000130000009300F000AF
:1004E0003B8720021302120093022000E31252FE07
:1004F0009303500A93019001631C77049300F00169
:100500003B011002930300009301A00163127104E8
:10051000930000023B810002930300009301B001AD
:1005200063187102BB000002930300009301C00135
:100530006390700293001002130120023B8020029E
:10054000930300009301D001631470006310300224
:100550000F00F00F638001009391110093E11100EF
:100560009308D00513850100730000000F00F00F01
:10057000930110009308D0051305000073000000DC
:10058000731000C000000000000000000000000028
:10059000000000000000000000000000000000005B
:1005A000000000000000000000000000000000004B
:0C05B0000000000000000000000000003F
:1010000000000000000000000000000000000000E0
:1010100000000000000000000000000000000000D0
:1010200000000000000000000000000000000000C0
:1010300000000000000000000000000000000000B0
:081040000000000000000000A8
:040000058000000077
:00000001FF
